:100000000C946E000C9403020C948B000C948B00E7
:100010000C948B000C948B000C948B000C948B0034
:100020000C948B000C948B000C948B000C948B0024
:100030000C948B000C948B000C948B000C948B0014
:100040000C948B000C948B000C948B000C948B0004
:100050000C948B000C948B000C948B000C948B00F4
:100060000C948B000C948B0009022200010100A06B
:100070000A09040000010300000009210101000138
:100080002216000705810308006412011001000018
:100090000008C016DF05000101020001140344003E
:1000A000610074006100530074006F00720065000D
:1000B00012036F0062006400650076002E0061008C
:1000C0007400040309040600FF0901A101150026BC
:1000D000FF00750895800900B20201C011241FBEFF
:1000E000CFEFD4E0DEBFCDBF11E0A0E0B1E0E0E7AC
:1000F000F7E002C005900D92A230B107D9F721E0D8
:10010000A2E0B1E001C01D92AB33B207E1F70E945B
:1001100070030C94B6030C940000CF93C62F20916B
:10012000100124FF19C02091110138E823272093E2
:1001300011012C2FFC01A2E1B1E081918D9321509E
:100140001216DCF36C2F82E191E00E94FF01CC5F7C
:10015000C0931001CF9108952AE520931001E9CFB3
:10016000CF93DF9360912101635067FDACC0809114
:100170001E01CCE0D0E0C81BD109CB5DDE4F8091E1
:100180001D018D3209F0DDC0683009F09AC083ECA2
:10019000809305018AE58093010110920201888114
:1001A000807679F0CE010E945E038F3F09F481C012
:1001B0009F81911184C09E81981708F080C0892F7B
:1001C0007EC02A8110920E01998191110AC010926D
:1001D0000F012EE031E082E03093200120931F01D7
:1001E000E7CF953029F4209322012EE031E0F4CFBF
:1001F000963009F047C09B81913041F48AE890E045
:100200009093200180931F0182E109C0923059F43C
:1002100088E690E09093200180931F0182E290E4B1
:1002200090930201C5CF9330C9F4211108C082EC2C
:1002300090E09093200180931F0184E0F0CF213063
:1002400019F480EB90E0DCCF223049F78CE990E0A4
:100250009093200180931F0184E1E1CF913241F41A
:100260008AE790E09093200180931F0189E0D7CF27
:100270009232A9F686EC90E09093200180931F01C2
:1002800086E1CDCF983071F0993019F42093240194
:10029000ACCF9A3059F09B3009F0A7CF9BE49093F4
:1002A0001101A3CF24E231E081E096CF2EE031E0CE
:1002B000FBCF988197FD8E8190E890930201809307
:1002C0000001109221018091010184FF2DC08091D5
:1002D00000018F3F49F1C82F893008F0C8E08C1B1E
:1002E000809300018091050198E88927809305019A
:1002F000CC2369F08091020187FF36C06C2F86E025
:1003000091E00E942403C82F893008F051C06C2F5F
:1003100086E091E00E94FF01CC5FCC3019F08FEFB6
:1003200080930001C093010184E199B1947131F48B
:100330008150D9F71092220110921C01DF91CF91C8
:1003400008958091020187FFBCCFCE010E943E0339
:100350008F3F21F48EE180930101B3CF882309F40C
:10036000B0CF10920001ADCF40911F0150912001FC
:1003700086FF15C0A6E0B1E0FA019C2F84918D9311
:1003800031969150D9F72FEF2C0F30E02F5F3F4F70
:10039000240F351F3093200120931F01B8CFDA01BD
:1003A000E6E0F1E09C2F8D9181939150E1F7EBCF46
:1003B0008FEF80930001CEE1B5CFE9E6F0E08081D8
:1003C00082608083E89AE0E1F1E08BE481838AE552
:1003D00080830895A82FB92F80E090E041E050EA93
:1003E000609530E009C02D9182279795879510F090
:1003F00084279527305EC8F36F5FA8F30895EADF7E
:100400008D939D930895CF93CFB7CF93DF93C395EB
:100410004C9BE9F74C9B0BC04C9B09C04C9B07C005
:100420004C9B05C04C9B03C04C9B01C08BC06F9381
:10043000C0911E01DD27CB5DDE4F2F9365E54C9B00
:1004400003C02F916F91E6CF0F931F934F9320E03E
:1004500040E15F9309B1047104FB27F93F9350E039
:100460003BE039C0147140642F77012F5F5F1EC0DD
:10047000406819B114712F7752501FC0406409B100
:100480002F770471D1F15F5F00C023C0406219B1C2
:100490002F77147191F15F5F00C025C004711027A0
:1004A000515012F45D5F0000115027952C3F19B197
:1004B000C8F614710127015027952C3FC8F6422732
:1004C000499309B1047110274F73115027952C3FA0
:1004D000A8F64695469519B1147179F00127015097
:1004E00027952C3F98F66B5A60F3315009B1B0F65E
:1004F00000C011E01CBB002719C03B503195C31B45
:10050000D04011E01CBB0881033C09F10B34F9F029
:1005100020911C011981110F1213EDCF4A81441F44
:10052000093651F10D3211F0013E29F700932301F4
:100530003F915F914F911F910F912F916F91CCB38C
:10054000C0FD65CFDF91CF91CFBFCF91189520919E
:100550002301222369F310912101112391F53430F5
:1005600092F13093210120931D0110911E013BE077
:10057000311B30931E0127C00091210101300CF581
:100580000AE54F7049F43091010134FD1DC000931C
:100590000101C5E0D1E01CC03091100134FD14C050
:1005A00000931001C1E1D1E013C0052710E000C0A5
:1005B00000000BB91AC0052710E0221F1DC010E073
:1005C00021C04AE502C032ED432FC4E1D0E032E061
:1005D0001AB114615C9A0BB11AB954E120E865E3D1
:1005E00020FF05270BB9279517951C3FF0F6669558
:1005F000B8F7B1F720FF05270BB9279517951C3FD2
:10060000D0F62795179517FF052700001C3F0BB95B
:10061000B0F629913A9519F70B7E10912201110F2E
:10062000C651D0400BB911F010931C0111E01CBB56
:1006300000611AB11B7E402F4B7E54E05A95F1F7B2
:100640000BB91AB94BB974CFCF93C09103016C1792
:1006500008F4C62F4C2F50E06091040170E00E9416
:100660008E03809104018C0F80930401809103011B
:100670008C1B809303018C2FCF910895CF93C09151
:100680000301CC23C9F06C1708F4C62F4C2F50E09F
:100690006091040170E00E949E03809104018C0F20
:1006A00080930401909103019C1B9093030181E0CE
:1006B000911180E0CF91089581E0FCCFFC01908101
:1006C0009076903259F48181877F813039F480E8C7
:1006D00080930301109204018FEF089580E0089544
:1006E0009EE088E10FB6F894A895809360000FBE55
:1006F000909360000E94DD01549A80E0815031F4B3
:1007000054987894A8950E94B000FCCFA895EFE982
:10071000FFE03197F1F700C00000F0CFDC01CB0122
:10072000FC01F999FECF06C0F2BDE1BDF89A319601
:1007300000B40D9241505040B8F70895DC01CB0150
:1007400003C02D910E94A90341505040D0F7089555
:10075000262FF999FECF1FBA92BD81BD20BD0FB6DD
:10076000F894FA9AF99A0FBE01960895F894FFCF7B
:02077000FF5A2E
:00000001FF
